:020000040800F2
:100000005008002089010008411A0008431A00081E
:10001000471A00084B1A00084F1A00080000000099
:10002000000000000000000000000000531A00085B
:10003000551A000800000000571A0008591A000855
:100040009F0100089F0100089F0100089F01000810
:100050009F0100089F0100089F0100089F01000800
:100060009F0100089F0100089F0100089F010008F0
:100070009F0100089F0100089F0100089F010008E0
:100080009F0100089F0100089F0100089F010008D0
:100090009F0100089F0100089F0100089F010008C0
:1000A0009F0100089F0100089F0100089F010008B0
:1000B0009F0100089F0100089F0100089F010008A0
:1000C0009F0100089F0100089F0100089F01000890
:1000D0009F010008051600089F0100089F01000805
:1000E0009F0100089F0100089F01000800F002F82E
:1000F00000F03AF80AA090E8000C82448344AAF188
:100100000107DA4501D100F02FF8AFF2090EBAE885
:100110000F0013F0010F18BFFB1A43F0010318473B
:10012000C4230000E4230000103A24BF78C878C13B
:10013000FAD8520724BF30C830C144BF04680C60ED
:10014000704700000023002400250026103A28BF35
:1001500078C1FBD8520728BF30C148BF0B60704739
:100160001FB51FBD10B510BD01F04FFE1146FFF7C2
:10017000F7FF01F015FC01F06DFE03B4FFF7F2FF8D
:1001800003BC01F0CBF9000008480047FEE7FEE79A
:10019000FEE7FEE7FEE7FEE7FEE7FEE7FEE7FEE737
:1001A00003480449044A054B70470000ED0000086D
:1001B000500200205008002050040020500400206D
:1001C00031490143314A1160704770B50021002365
:1001D0000F22C47804B32D4C246804F4E064C4F501
:1001E000E064210AC1F10403CA40447804FA03F12F
:1001F0008478144021430901254C0678A1550478E0
:1002000004F01F050124AC4005786D11AD0005F127
:10021000E025C5F8004109E0047804F01F05012439
:10022000AC401C4D0678761145F8264070BD1A4A40
:100230000A400243154B1B1F1A60704739B1134A1D
:10024000121D12680243114B1B1D1A6006E00F4A73
:10025000121D126882430D4B1B1D1A607047042843
:1002600008D14FF0E021096941F004014FF0E0228C
:10027000116107E04FF0E021096921F004014FF01E
:10028000E0221161704700000000FA050CED00E06B
:1002900000E400E080E100E080FFFF1F10B50446AD
:1002A000FA48844208D10121401500F055FD002193
:1002B000601500F051FD17E0F548844208D1012196
:1002C000001500F049FD0021201500F045FD0BE070
:1002D000F048844208D10121C80300F03DFD00210F
:1002E0004FF4004000F038FD10BD30B5024600204C
:1002F00000235068E84C20400D790C6844EA05243E
:10030000204350609068E54C2040D1E902542C43D2
:100310004D7944EA450420439060D06A20F470008F
:100320000C7C641EE4B2234340EA0350D06230BD2B
:1003300000210160017141718160C160012101747E
:10034000704721B1826842F00102826003E0826856
:1003500022F001028260704721B1826842F480720B
:10036000826003E0826822F480728260704710B578
:100370000023CBB21AB144681C43446002E04468D5
:100380009C43446010BD816841F008018160704762
:10039000014600208A6802F008020AB1012000E04C
:1003A00000207047816841F0040181607047014678
:1003B00000208A6802F004020AB1012000E0002057
:1003C000704721B1826842F4A002826003E0826833
:1003D00022F4A00282607047014600208A6802F47D
:1003E00080020AB1012000E00020704710B50A46E3
:1003F00000210023416821F46041531E41EA43314A
:10040000416010BD21B1426842F40062426003E0E5
:10041000426822F4006242607047F0B504460D461F
:1004200000200021092D11DDE068A5F10A0606EB88
:100430004607072606FA07F18843A5F10A0606EBE8
:10044000460603FA06F10843E0600CE0206905EB7C
:100450004507072606FA07F1884305EB450603FA28
:1004600006F108432061072A0FDA606B561E06EB7F
:1004700086071F2606FA07F18843561E06EB8606F6
:1004800005FA06F10843606322E00D2A0FDA206BBB
:10049000D61F06EB86071F2606FA07F18843D61FEC
:1004A00006EB860605FA06F10843206310E0E06AD1
:1004B000A2F10D0606EB86071F2606FA07F1884310
:1004C000A2F10D0606EB860605FA06F10843E06286
:1004D000F0BD21B1826842F48012826003E082683C
:1004E00022F48012826070470146C86C80B2704767
:1004F00066484C300068704721B1426842F480621F
:10050000426003E0426822F480624260704721B199
:10051000426842F48052426003E0426822F4805212
:10052000426070470A460021816821F4E04111438E
:100530008160704721B1826842F40042826003E02A
:10054000826822F400428260704721B1826842F4DE
:100550000212826003E0826822F402128260704715
:10056000014600208A6802F400120AB1012000E06E
:1005700000207047F0B504461546002000220026F2
:10058000092911DDE068A1F10A0707EB470C0727ED
:1005900007FA0CF29043A1F10A0707EB470703FAA9
:1005A00007F21043E0600CE0206901EB410C0727E3
:1005B00007FA0CF2904301EB410703FA07F21043EC
:1005C0002061A06BC0F30156EF1C06F1010CA7EBF4
:1005D0000C0707EB870C1F2707FA0CF29043EF1C60
:1005E00006F1010CA7EB0C0707EB870701FA07F2EE
:1005F0001043A063F0BD10B50A4600210023816BB3
:1006000021F44011531E41EA0351816310BD08B526
:10061000002300930090009B0B440093009B1A6002
:1006200008BD08B5024600200090009201F12800A4
:10063000009B184400900098006880B208BD0A46EC
:1006400000214168164B19401143416070474162D7
:10065000826270470A460021416821F01F01114360
:100660004160704740B109490831096841F400010F
:10067000064A0832116007E004490831096821F48C
:100680000001024A08321160704700000024014056
:1006900000280140003C0140FFFEF0FFFDF7F1FFA4
:1006A000FFFD3FFF0246002013680B400BB1012005
:1006B00000E000207047CA430260704770B50246F0
:1006C0000020002300240B125568CEB205EA060470
:1006D00015681D4015B10CB1012000E0002070BD6F
:1006E00000220A12D34303607047000010B504468D
:1006F000CC48844208D10121042000F02DFB0021C8
:10070000042000F029FB46E0C748844208D10121BB
:10071000082000F021FB0021082000F01DFB3AE03A
:10072000C248844208D10121102000F015FB0021AD
:10073000102000F011FB2EE0BD48844208D10121B9
:10074000202000F009FB0021202000F005FB22E022
:10075000B848844208D10121402000F0FDFA002170
:10076000402000F0F9FA16E0B348844208D1012194
:10077000802000F0F1FA0021802000F0EDFA0AE07C
:10078000AE48844207D10121801500F0E5FA00212E
:10079000A01500F0E1FA10BD10B50121084600F0E7
:1007A000DBFA0021012000F0D7FA10BD2DE9F0415D
:1007B000024600250026002000230024002791F88F
:1007C00003C00CF00F0591F803C00CF0100CBCF145
:1007D000000F03D091F802C04CEA050591F800C063
:1007E000BCF1000F31D0146800202BE04FF0010C59
:1007F0000CFA00F3B1F800C00CEA03069E4220D1C7
:1008000083004FF00F0C0CFA03F7BC4305FA03FC0E
:100810004CEA040491F803C0BCF1280F06D14FF054
:10082000010C0CFA00FCC2F814C00AE091F803C0F5
:10083000BCF1480F05D14FF0010C0CFA00FCC2F8D6
:1008400010C0401C0828D1D31460B1F800C0BCF11E
:10085000FF0F34DD546800202EE000F1080C4FF04B
:10086000010808FA0CF3B1F800C00CEA03069E4236
:1008700021D183004FF00F0C0CFA03F7BC4305FAAB
:1008800003FC4CEA040491F803C0BCF1280F05D125
:1008900000F1080C08FA0CF8C2F8148091F803C0B3
:1008A000BCF1480F07D100F1080C4FF0010808FA1D
:1008B0000CF8C2F81080401C0828CED35460BDE864
:1008C000F0814FF6FF710180022181700421C17017
:1008D00070470246002093680B400BB1012000E0F6
:1008E000002070470146886880B2704702460020A9
:1008F000D3680B400BB1012000E000207047014697
:10090000C86880B2704701617047416170470AB1A1
:10091000016100E041617047C16070474FF480326F
:100920000A438261816182618269826970470246FD
:100930000020434B18684FF68073184040EA0210BD
:1009400008433F4B186070473E49C8617047F0B597
:100950000A46002300240021002500F00046B6F1DD
:10096000004F02D1364EF16901E0354E7168C0F397
:10097000034583B200F44016B6F5401F08D121F0BC
:1009800070612F4E766826F070662D4F7E6012E003
:1009900000F48016B6F5801F06D1032606FA05F48A
:1009A000A14341F0706106E0460D360103FA06F6F8
:1009B000B14341F0706122B1460D360103FA06F6EB
:1009C000314300F00046B6F1004F02D11C4EF161F8
:1009D00001E01B4E7160F0BD30B500228B071C0F8B
:1009E0000F2303FA04F2164B08338C1053F824300B
:1009F0009343134C08348D1044F8253023468C1053
:100A000053F824308C07240F00FA04F423430C4CD1
:100A100008348D1044F8253030BD0A49DC310860B7
:100A20007047000000080140000C01400010014028
:100A30000014014000180140001C0140002001404A
:100A40000000014000002042DF48006840F0010043
:100A5000DD49086008464068DC490840DA494860DA
:100A600008460068DA490840D74908600846006827
:100A700020F4802008600846406820F4FE004860AA
:100A80004FF41F0088607047CF49096821F4803116
:100A9000CD4A11601146096821F480211160B0F53A
:100AA000803F03D0B0F5802F0ED106E0C64909681B
:100AB00041F48031C44A116007E0C349096841F438
:100AC000A021C14A116000E000BF00BF704710B50F
:100AD00001460022002300204A11012A02D1BA4C0B
:100AE000236806E0022A02D1B74C236A01E0B64C23
:100AF000636A01F01F02012494401C400CB10120E4
:100B000000E0002010BD38B5002000900024002532
:100B100000BF3120FFF7DBFF05460098401C009026
:100B20000098B0F5A06F01D0002DF2D03120FFF772
:100B3000CEFF08B1012400E00024204638BD014664
:100B40000020A14A106820F0F80040EAC1001060BF
:100B50007047A04908607047024600209A4B5868C9
:100B600020F47C1042EA01031843974B5860704709
:100B700098490866704701460020934A506820F063
:100B800003000843506070478F48406800F00C0035
:100B90007047014600208C4A506820F0F00008435E
:100BA0005060704701460020874A506820F4E0609A
:100BB00008435060704701460020834A506820F483
:100BC000605040EAC1005060704729B17E4A527AB5
:100BD00002437D4B5A7204E07B4A527A82437A4B3D
:100BE0005A7270477B49D83108607047014600202F
:100BF000754A506820F44040084350607047002117
:100C0000714A20321170704A82F82010012802D0F7
:100C100004280AD104E001216B4A2032117005E05A
:100C20000521694A2032117000E000BF00BF704703
:100C30006949086070476449096A0143624A116260
:100C40007047654944390860704730B5002100227B
:100C5000002400235C4D6D6805F00C0121B10429CE
:100C600005D0082923D105E05C4D056022E05B4DED
:100C700005601FE0544D6D6805F47012524D6D68AB
:100C800005F48034022505EB92421CB9544D5543BE
:100C900005600BE04C4D6D6805F400351DB1504DFD
:100CA0005543056002E04D4D5543056002E04B4D54
:100CB000056000BF00BF444D6D6805F0F0010909F3
:100CC000484D6B5C0568DD4045603F4D6D6805F43F
:100CD000E061090A434D6B5C4568DD4085603A4D33
:100CE0006D6805F46051C90A3E4D6B5C4568DD4096
:100CF000C560354D6D6805F44041890B3A4D6B5C1C
:100D0000C568B5FBF3F5056130BD29B12E4A5269BE
:100D100002432D4B5A6104E02B4A526982432A4B0D
:100D20005A61704729B1284A92690243264B9A6159
:100D300004E0254A92698243234B9A61704729B1A6
:100D4000214AD2690243204BDA6104E01E4AD2698B
:100D500082431D4BDA61704729B11B4AD2680243B6
:100D6000194BDA6004E0184AD2688243164BDA6005
:100D7000704729B1144A12690243134B1A6104E007
:100D8000114A12698243104B1A6170471249403967
:100D9000086070470F49C86470470B49C8717047B5
:100DA0000948406A40F08070074948627047014630
:100DB0000020054A92680A400AB1012000E00020A4
:100DC0007047014988727047001002400000FFF828
:100DD000FFFFF6FE000042428004424200127A0009
:100DE00000093D00000000201000002010B504465E
:100DF000FB48844209D101218803FFF7ADFF0021A0
:100E00004FF48040FFF7A8FF32E0F648844209D152
:100E100001214804FFF7ADFF00214FF40030FFF738
:100E2000A8FF25E0F048844209D101218804FFF79A
:100E3000A0FF00214FF48020FFF79BFF18E0EB4854
:100E4000844209D10121C804FFF793FF00214FF428
:100E50000020FFF78EFF0BE0E548844208D1012116
:100E60000805FFF786FF00214FF48010FFF781FF90
:100E700010BD2DE9F04786B005460E460024A24677
:100E800000BFA1460027B08900B100BF2F462C8AC1
:100E90004CF6FF700440F08804432C82AC894EF677
:100EA000F3100440B0883189084371890843044332
:100EB000AC81AC8A4FF6FF400440B0890443AC8259
:100EC00001A8FFF7C2FEC648874202D1DDF810A094
:100ED00001E0DDF80CA0A88900F4004040B10AEB65
:100EE000CA0000EB0A1031684900B0FBF1F807E0D6
:100EF0000AEBCA0000EB0A1031688900B0FBF1F878
:100F00006420B8FBF0F004012009642101FB108982
:100F1000A88900F4004040B1322000EBC900B0FBCA
:100F2000F1F000F00700044308E0322000EB091064
:100F30006421B0FBF1F000F00F0004432C8106B0F7
:100F4000BDE8F0874FF41651016000218180C18017
:100F500001810C21418100218181704710B5024639
:100F60000020108A4FF2FF0318400B884C8823435F
:100F70008C882343CC8823431843108210BD002162
:100F8000018041808180C180704721B1828942F413
:100F90000052828104E082894DF6FF731A408281FB
:100FA0007047F0B50346002400260025002040F6D7
:100FB0006A17B94200D100BF1846C1F3421401F0CC
:100FC0001F06012707FA06F5012C01D10C3004E0B9
:100FD000022C01D1103000E014301AB107682F4301
:100FE000076002E00768AF430760F0BD1AB1838A6B
:100FF0000B43838202E0838A8B4383827047028A99
:101000004FF6F0731A400282028A0A430282704746
:1010100082894FF2FF731A40828182890A4382815A
:10102000704721B1828942F00202828104E0828904
:101030004FF6FD731A4082817047028A4FF6DF73C4
:101040001A400282028A0A430282704721B1028A50
:1010500042F48042028204E0028A4BF6FF731A4097
:1010600002827047C1F30802828070470146888877
:10107000C0F308007047818941F001018181704708
:10108000028BD2B20283028B42EA012202837047B2
:10109000028B02F47F420283028B0A430283704771
:1010A00021B1828A42F02002828204E0828A4FF6D5
:1010B000DF731A408282704721B1828A42F01002A7
:1010C000828204E0828A4FF6EF731A408282704770
:1010D00021B1828A42F00802828204E0828A4FF6BD
:1010E000F7731A408282704721B1828942F400422C
:1010F000828103E08289C2F30E028281704721B1AE
:10110000828A42F40062828204E0828A4FF2FF7394
:101110001A4082827047828A4FF6FB731A4082829D
:10112000828A0A438282704721B1828A42F0020297
:10113000828204E0828A4FF6FD731A4082827047F1
:1011400002460020B1F5007F00D100BF13880B409C
:101150000BB1012000E00020704701F40072B2F5ED
:10116000007F00D100BFCA430280704770B50246BD
:10117000002400230025002040F66A16B14200D169
:1011800000BFC1F3421501F01F03012606FA03F365
:10119000012D02D19689334006E0022D02D1168A34
:1011A000334001E0968A33400C12012606FA04F41B
:1011B0001688344013B10CB1012000E0002070BD4E
:1011C00010B50022002340F66A14A14200D100BFEE
:1011D0000A1201249440A3B2DC43048010BD000035
:1011E000003801400044004000480040004C0040EE
:1011F0000050004001684FF6FE721140016000216E
:10120000016041608160C1608D49884208D18C498C
:101210000839496841F00F01894A083A51608AE06B
:1012200087491431884208D185490839496841F015
:10123000F001834A083A51607DE0814928318842B3
:1012400008D17F490839496841F470617C4A083AFD
:10125000516070E07A493C31884208D178490839B8
:10126000496841F47041764A083A516063E0744934
:101270005031884208D172490839496841F47021D7
:101280006F4A083A516056E06D496431884208D18E
:101290006B490839496841F47001694A083A51605C
:1012A00049E067497831884208D165490839496879
:1012B00041F07061624A083A51603CE061498842FD
:1012C00006D1011F096841F00F01021F116032E0D1
:1012D0005C491431884208D15A49091F096841F014
:1012E000F001584A121F116025E056492831884202
:1012F00008D15449091F096841F47061514A121F0D
:10130000116018E04F493C31884208D14D49091F0E
:10131000096841F470414B4A121F11600BE04949C2
:101320005031884207D14749091F096841F47021AB
:10133000444A121F1160704710B50022026847F638
:10134000F0739A430C6A8B6823430C6923434C69FE
:1013500023438C692343CC6923434C6A23438C6A1F
:1013600023431A430260CB6843600B6883604B6879
:10137000C36010BD0021016041608160C1600161F6
:1013800041618161C161016241628162704721B145
:10139000026842F00102026004E002684FF6FE7348
:1013A0001A40026070471AB103680B43036002E001
:1013B00003688B430360704741607047014648688B
:1013C00080B2704701460020002201F080531BB11B
:1013D0001C4B083B1A6802E0194B083B1A6802EAEA
:1013E00001030BB1012000E00020704700F08051A4
:1013F00019B11449091F086002E011490839486011
:10140000704701460020002201F080531BB10D4BB4
:10141000083B1A6802E00A4B083B1A6802EA01031B
:101420000BB1012000E00020704700F0805119B19D
:101430000449091F086002E0014908394860704703
:10144000080002400804024010B56FF00400FEF7E7
:1014500006FF2E4800682E49B0FBF1F02D490870B8
:101460000846007800EB4001C1EBC0104FF6FF7159
:1014700001EAC0002849088010BD0146254A1278BB
:101480004A434FF0E0235A6100229A611A461269DA
:1014900042F001021A6100BF4FF0E022106900F033
:1014A00001021AB100F48032002AF5D04FF0E02298
:1014B000126922F001024FF0E0231A6100229A61C2
:1014C00070470146144A12884A434FF0E0235A619C
:1014D00000229A611A46126942F001021A6100BFA5
:1014E0004FF0E022106900F001021AB100F48032DE
:1014F000002AF5D04FF0E022126922F001024FF0ED
:10150000E0231A6100229A61704700002000002049
:1015100000127A001400002016000020014600BFCF
:10152000704700BF564A128802F04002002AF9D0E4
:10153000C2B2534B1B1D1A80704710B586B00446CB
:10154000012144F20400FFF7EDFB4FF40070ADF809
:10155000140003208DF8160018208DF8170005A937
:101560004848FFF723F94FF48060ADF814000420D9
:101570008DF8170005A94348FFF718F925208DF8C5
:10158000000003208DF801008DF8020001208DF885
:1015900003006846FEF719FE01940020ADF808002C
:1015A000ADF80A00ADF80C00ADF810000C20ADF855
:1015B0000E0001A93248FFF75CFC012240F22551E0
:1015C0002F48FFF7EEFC01212D48FFF7DEFC06B0A7
:1015D00010BD10B5044621462948FFF743FD00BF62
:1015E00040212748FFF7ACFD0028F9D010BD10B509
:1015F000044603E014F8010BFFF7EBFF2078002806
:10160000F8D110BD10B540F225511D48FFF7AEFDD1
:1016100010B31B48FFF72AFDC4B21B48008800F432
:101620000040C8B91848008800F4804060B10A2C16
:1016300003D000201449088020E01348008840F4BB
:1016400000401149088019E00D2C06D10E48008891
:1016500040F480400C49088010E00B480088C0F33B
:101660000D000A490C5408480088401C06490880AF
:1016700008460088C72801DD0020088010BD000052
:1016800000380140000801401C0000203400002008
:101690002DE9F04104464FF47A7094FBF0F0C5B2A6
:1016A000642094FBF0F00A2190FBF1F201FB1200A0
:1016B000C6B20A2094FBF0F090FBF1F201FB12009D
:1016C000C7B20A2094FBF0F100FB114000F0FF08C4
:1016D00005F13001C8B2FFF77CFF06F13001C8B256
:1016E000FFF777FF07F13001C8B2FFF772FF08F18B
:1016F0003001C8B2FFF76DFFBDE8F0812DE9FE4F64
:101700008246504600F08EFD009000F0DDFC07465A
:101710004FF06632B24B00F0D9FB054600F0A4FB57
:101720000446204600F05EFD1FFA80F909F1300101
:10173000C8B2FFF74EFF484600F074FD054621464B
:1017400000F050FE0446A749204600F07FFD044605
:10175000204600F047FD80B2642190FBF1F080B29A
:101760000290204600F03EFD80B2642190FBF1F231
:1017700001FB12000A2190FBF1F080B2019020469B
:1017800000F030FD80B20A2190FBF1F201FB120063
:101790001FFA80FB2E20FFF71CFF02993031C8B2E0
:1017A000FFF717FF01993031C8B2FFF712FF0BF1B5
:1017B0003001C8B2FFF70DFFBDE8FE8F10B58AA05B
:1017C000FFF715FF002000F0CCFA0446FFF760FF9A
:1017D0000920FFF7FEFE002000F0C3FA0446FFF7E1
:1017E0008DFF5620FFF7F5FE81A0FFF700FF81A0D7
:1017F000FFF7FDFE012000F0B4FA0446FFF748FFB2
:101800000920FFF7E6FE012000F0ABFA0446FFF7DF
:1018100075FF5620FFF7DDFE75A0FFF7E8FE77A005
:10182000FFF7E5FE022000F09CFA0446FFF730FFC8
:101830000920FFF7CEFE022000F093FA0446FFF7DE
:101840005DFF5620FFF7C5FE69A0FFF7D0FE6DA033
:10185000FFF7CDFE032000F084FA0446FFF718FFDF
:101860000920FFF7B6FE032000F07BFA0446FFF7DD
:1018700045FF5620FFF7ADFE5DA0FFF7B8FE63A061
:10188000FFF7B5FE042000F06CFA0446FFF700FFF6
:101890000920FFF79EFE042000F063FA0446FFF7DC
:1018A0002DFF5620FFF795FE51A0FFF7A0FE59A08F
:1018B000FFF79DFE052000F054FA0446FFF7E8FE0E
:1018C0000920FFF786FE052000F04BFA0446FFF7DB
:1018D00015FF5620FFF77DFE45A0FFF788FE4FA0BD
:1018E000FFF785FE062000F03CFA0446FFF7D0FE25
:1018F0000920FFF76EFE062000F033FA0446FFF7DA
:10190000FDFE5620FFF765FE39A0FFF770FE45A0EB
:10191000FFF76DFE072000F024FA0446FFF7B8FE3B
:101920000920FFF756FE072000F01BFA0446FFF7D8
:10193000E5FE5620FFF74DFE2DA0FFF758FE3BA019
:10194000FFF755FE082000F00CFA0446FFF7A0FE52
:101950000920FFF73EFE082000F003FA0446FFF7D7
:10196000CDFE5620FFF735FE21A0FFF740FE31A047
:10197000FFF73DFE092000F0F4F90446FFF788FE6A
:101980000920FFF726FE092000F0EBF90446FFF7D7
:10199000B5FE5620FFF71DFE15A0FFF728FE10BD6F
:1019A00000F0CBF8FFF750FD4FF4A060FEF708FC05
:1019B0004FF4E130FFF7C1FD00F040F90FE000BF48
:1019C00080211E48FFF7BCFB0028F9D0FFF7F6FE88
:1019D00007A0FFF70CFE4FF4FA70FFF772FDEEE779
:1019E00066664A3F00007A444348303A00000000EF
:1019F0000D0A00004348313A000000004348323AE3
:101A0000000000004348333A000000004348343AE5
:101A1000000000004348353A000000004348363AD1
:101A2000000000004348373A000000004348383ABD
:101A3000000000004348393A00000000003801402F
:101A4000704700BFFEE700BFFEE700BFFEE700BF34
:101A5000FEE7704770477047704700000CB50020E4
:101A6000019000906C48006840F480306A4908603A
:101A700000BF6948006800F4003000900198401CE5
:101A80000190009818B90198B0F5A06FF1D16248A3
:101A9000006800F4003010B10120009001E0002047
:101AA00000900098012843D15C48006840F0100085
:101AB0005A4908600846006820F00300086008469C
:101AC000006840F00200086053484068524948608E
:101AD0000846406848600846406840F480604860B6
:101AE0000846406820F47C1048600846406840F48E
:101AF000E81048600846006840F08070086000BF49
:101B00004548006800F000700028F9D0424840685D
:101B100020F00300404948600846406840F0020059
:101B2000486000BF3C48406800F00C000828F9D12C
:101B30000CBD10B5FFF792FF10BD10B53648006818
:101B400040F00100344908600846406834490840C4
:101B50003149486008460068324908402E4908600B
:101B60000846006820F4802008600846406820F499
:101B7000FE0048604FF41F008860FFF7DAFF4FF067
:101B800000602949086010BD10B500210020002226
:101B9000214B5B6803F00C0121B1042906D0082910
:101BA00028D107E0214B224C236027E01F4B204C1B
:101BB000236023E0184B5B6803F47010164B5B68DE
:101BC00003F48032022303EB904022B9194B4343C4
:101BD000174C23600DE0104B5B6803F4003323B116
:101BE000144B4343124C236003E0104B4343104C0F
:101BF000236003E00D4B0E4C236000BF00BF064B7B
:101C00005B68C3F303130C4CE15C094B1B68CB40CE
:101C1000074C236010BD000000100240002002406D
:101C20000000FFF8FFFFF6FE08ED00E000127A006A
:101C30002000002000093D002400002000B587B0EE
:101C400001214FF40370FFF76DF84FF40040FEF7E9
:101C5000CDFFFF20ADF8040000208DF8070001A99A
:101C60004B48FEF7A3FD0320ADF8040000208DF8DB
:101C7000070001A94748FEF799FD00F091F8464892
:101C8000FEF70CFB0020029001208DF80C008DF86F
:101C90000D004FF460200490002005900A208DF87C
:101CA000180002A93C48FEF720FB0723012200216F
:101CB0003948FEF7B2FB0723022201213648FEF71E
:101CC000ACFB0723032202213348FEF7A6FB0723C0
:101CD000042203213048FEF7A0FB0723052204213C
:101CE0002D48FEF79AFB0723062205212A48FEF716
:101CF00094FB07231A4606212748FEF78EFB07238D
:101D0000082219462448FEF788FB072309220821E8
:101D10002148FEF782FB07230A2209211E48FEF70D
:101D20007CFB01211C48FEF717FB01211A48FEF736
:101D300008FB1948FEF727FB00BF1748FEF728FBF2
:101D40000028FAD11448FEF72DFB00BF1248FEF719
:101D50002EFB0028FAD101210F48FEF732FB07B015
:101D600000BD10B502460023002109E001EB81000F
:101D70000A4C04EB800030F812000344481CC1B246
:101D80000A29F3DB0A20B3FBF0F080B210BD00009B
:101D900000080140000C014000240140FC0000202C
:101DA00010B501210846FEF7B0FF1148FFF722FAEF
:101DB000104811490860114848600020886064207C
:101DC000C860002008618020486140008861800070
:101DD000C86120200862000248620020886204482E
:101DE000FFF7AAFA01210248FFF7D1FA10BD00005F
:101DF000080002404C240140C4010020FC000020E7
:101E000070477047704770477047754600F028F874
:101E1000AE4605006946534620F00700854618B0D7
:101E200020B5FEF7BDF9BDE820404FF000064FF0A9
:101E300000074FF000084FF0000B21F00701AC46FF
:101E4000ACE8C009ACE8C009ACE8C009ACE8C0091E
:101E50008D4670470446AFF300802046FEF78DF9AB
:101E600000487047F001002021F00042A2F16052CA
:101E7000B2F5801F01F0004328BFD2F17F6C0BD96F
:101E80005FEA001C43EAC20242EB507018BF704781
:101E900028BF20F001007047B2F5801FBCBF184674
:101EA00070474FEA410C1CF5001F02D2084600F0B3
:101EB00094BA70B500F0B4F800000089FFF7F6BFDF
:101EC0004FF00040A0F5800070470000DFF848C1E7
:101ED00070B51CEA111E1EBF1CEA13159EEA0C0FFA
:101EE00095EA0C0F00F06F8081EA030423EA4C139B
:101EF0004EEAD47E21EA4C1141F4801143F4801360
:101F0000AE44A1FB024CA0FB0365AEF17F7E361907
:101F100055EB0C05A1FB034C4CF10003A0FB021C8C
:101F200016EB0C06654153F10003094218BF46F059
:101F3000010613F4007F0BD14FEA03314FEA05305D
:101F4000340341EA155140EA16506FF003020AE0EB
:101F50004FEAC3214FEAC520F40241EA555140EA55
:101F600056506FF0020202EB2E4201EB025585EA59
:101F7000CE710AD05FEA440C18BF24F0004450F13F
:101F8000000041F1000120EAD47040F2FE7C62457D
:101F900000D270BDA84214BF4FF080444FF04044BF
:101FA000002E08BF0024BEF1806FA8BFA1F1C04180
:101FB000BDE8704080F282804FF0000001F1C04126
:101FC00001F0004170479EEA0C0F0CEA131518BF90
:101FD00095EA0C0F06D04FF0000081EA030E0EF0D8
:101FE000004170BD00F01CF88900013E00F007B808
:101FF00000F009B84FEA430C5FEA5C5C08D081EA64
:10200000030100F05BB84FEA410C5FEA5C5CF6D17B
:102010004FF00000014970470000FF070000F87F03
:102020000EF1020E2EF0030E5EF8046B364205D45C
:10203000012A43EB030515F5001F12D8012841EBD7
:10204000010C1CF5001F0CD80ED14FEAD17C15F500
:10205000001F0CEB4C0C0CF1020C08BF4CEBD37CBA
:1020600004E04FF0080C01E04FEAD37C0CEB4C0588
:1020700026FA05F606F00706B6F1040C06D20EEBBA
:10208000860CBDE870404CF0010C6047DFE80CF0B6
:10209000090B02024FF000414FF00000A1F50021B2
:1020A00070BD19461046012851EB010418BFD4F544
:1020B000001484BF002001F0004170BD0808A0F5A5
:1020C00000114FEA3101704743004FEAD30C4FEA49
:1020D0003C0C43401FBF40070CF1605113F0FE4F12
:1020E00070471CF0006F03D100200CF000417047D6
:1020F0000CF0004343EA507010B540EACC0000F009
:1021000026F900BF000000924FEA0001FFF7D6BF9A
:102110004FF000414FF00000A1F500217047000092
:1021200090EA010F48BF81F0004100F16C81421A32
:102130003CBF801A89184FEAD0524FF07F4C1CEAFE
:10214000410FA2EBD15318BF9CEA026F00F03B8015
:102150004FF0004C4CEA00204CEA012121FA03FC2C
:1021600010EB0C0C1ED202F1FF325FEA1C2040EB98
:10217000C25038BF70471CF07F0F4FEA400C18BFA9
:10218000BCF17F4F38BF7047C3F12003994008BFAF
:1021900020F00100BCF17F4F38BF7047A0F1C04074
:1021A00000F01BB94FEA3C00000A40EBC25028BFC8
:1021B0001CF0FF0F4FEA400CE6D018BFBCF17F4F78
:1021C00038BF7047EAE79CEA026F05D010EA5C0F5F
:1021D00008BF00F00040704710B500F0B8F800BF2D
:1021E00064FBBE3EC10DD1F19E0206DB4FEA002327
:1021F00043F0004323FA02F07047004207D54FEA4C
:102200004001B1F1FE4F02D24FF00000704710B50F
:1022100000F09DF849922480002070476FEA20006A
:1022200070470000B0FA80F310FA03F2C3F19D0387
:102230000AD0D90501EB1220530638BF704700F1D0
:10224000010008BF20F00100704700004FF47F0C30
:102250001CEAD0121EBF1CEAD11392EA0C0F93EABB
:102260000C0F00F0478090EA010F48BF42F48072E3
:102270004FF0004C4CEA00204CEA012102EB030233
:10228000A0FB0113A2F50002002918BF43F00103CF
:102290005B0028BF4FEA330342EB22425FEA132C74
:1022A0004CEBC2502EBFBCEB436FB2F57C0F7047B6
:1022B0004FEA036CBCF1004F08BF20F00100B2F5FB
:1022C0007C0F38BF70470BD582F0FF0212F5803FBC
:1022D000C8BF704700F1C040D8BF00F00040704751
:1022E00000F5000C5FEA4C0C48BF7047B0F1C040ED
:1022F00000F073B890EA010F0CEAD11348BF42F422
:102300008072624538BF634504D280EA010000F064
:102310000040704710B500F01AF800BF8900013E78
:1023200000F007B800F009B85FEA410C5FEA1C6CE6
:1023300008D080EA010000F050B85FEA400C5FEA84
:102340001C6CF6D14FF00040A0F5800070470EF1F4
:10235000020E2EF0030E5EF8044B244204D44FEA22
:102360004102B2F17F4F11D84FEA4003B3F17F4FE2
:102370000CD80ED14FEAD07CB2F17F4F0CEB4C0C55
:102380000CF1020C08BF4CEBD17C04E04FF0080CC0
:1023900001E04FEAD17C0CEB4C0324FA03F404F087
:1023A0000704B4F1040C06D20EEB840CBDE8104017
:1023B0004CF0010C6047DFE80CF0070802024FF018
:1023C0000040A0F5800010BD0846420018BFD2F1C1
:1023D000807288BF00F0004010BDFF2141EAD0505C
:1023E000C005704780F0004090EA010F7FF59FAE76
:1023F00081F0004100F007B890EA010F48BF81F07A
:1024000000413FF594AE421A04D882F00042A0EB9E
:10241000020011444FEAD0524FF07F4C1CEA410FAA
:10242000A2EBD15318BF9CEA026F4AD04FF0004C88
:102430004CEA00204CEA012121FA03FCB0EB0C0C21
:102440000FD412F0FE0F36D05FEA4C001DD50012FB
:1024500040EBC25038BF70471CF03F0F18BF7047A9
:102460000BE0A2F101025FEA1C2040EBC25038BF32
:1024700070471CF07F0F18BF7047C3F120039940CD
:1024800014BF401E20F00100704780084FEA12235D
:1024900008BF7047B0FA80FCA2EB0C02CCF1280C0C
:1024A00060FA0CF093EA122F04BF00EBC2507047A1
:1024B0004FEAC3707047130A5FEADC1008BF704729
:1024C000F6E79CEA026F04D010EA5C0F08BF002018
:1024D000704710B5FFF73BFF40DFF63E81F000404C
:1024E00070470000042500080000002034000000B0
:1024F0002801000838250008340000201C080000CE
:10250000440100080000000001020304010203046A
:102510000607080902040608000000000000000089
:102520000000000000A24A040000000000000000BB
:0825300001020304060708097B
:04000005080000ED02
:00000001FF
